:100000000C9435000C945D000C945D000C945D0024
:100010000C945D000C945D000C945D000C945D00EC
:100020000C945D000C945D000C945D000C945D00DC
:100030000C945D000C945D000C945D000C945D00CC
:100040000C945D000C945D000C945D000C945D00BC
:100050000C945D000C945D000C945D000C945D00AC
:100060000C945D000C945D00210311241FBECFEFA2
:10007000D4E0DEBFCDBF11E0A0E0B1E0E4ECF6E0FB
:1000800002C005900D92AA38B107D9F723E0AAE87B
:10009000B1E001C01D92AF31B207E1F710E0CAE64E
:1000A000D0E004C02297FE010E945C03C836D1074D
:1000B000C9F70E94A3020C9460030C94000020E096
:1000C00030E080E061E070E04A99FECF289AE7EBEB
:1000D000FBE03197F1F700C000004A9908C0AB017E
:1000E000022E02C0440F551F0A94E2F7842B4A9B4C
:1000F000FECF2898F2E4FA95F1F700C02F5F3F4F4A
:100100002830310509F708951F93CF93DF934A995B
:1001100016C28FE19EE40197F1F700C000004A99F2
:100120000EC24A9BFECF0E945F00182F0E945F0004
:100130000E945F00482FC82FD0E0E0ECF0E0808103
:1001400085FFFDCF80E38093C60060E070E0CB01C7
:100150009695879596958795969587959C01220FFC
:10016000331F880F991F880F991F880F991F820FBF
:10017000931F681B790B605DE0ECF0E0808185FFE8
:10018000FDCF6093C6009E0136952795369527953D
:10019000ABE7B4E10E944E0396958795805DE0EC55
:1001A000F0E0908195FFFDCF8093C6009E01ADECFD
:1001B000BCEC0E944E03FC01F695E795F695E79599
:1001C000F695E7959F010E944E0396958795969523
:1001D0008795969587959C01220F331F880F991F4D
:1001E000880F991F880F991F820F931FE81BF90B27
:1001F0009E2F905DE0ECF0E0808185FFFDCF909335
:10020000C6009E01ADECBCEC0E944E03969587950E
:1002100096958795969587959C01220F331F880F99
:10022000991F880F991F880F991F820F931FC81B52
:10023000D90BC05DE0ECF0E0808185FFFDCFC0937D
:10024000C600A4E5B1E090E2E0ECF0E0C6ECD0E05E
:10025000808185FFFDCF98839D919111F9CFE0ECCE
:10026000F0E0808185FFFDCF8DE08093C600E0EC5B
:10027000F0E0808185FFFDCF8AE08093C6001111F8
:100280005EC14F3E09F05BC10E945F00182F0E94C3
:100290005F00482FABE5B1E022E5E0ECF0E0C6EC12
:1002A000D0E0908195FFFDCF28832D912111F9CFCA
:1002B000E0ECF0E0908195FFFDCF8DE08093C600EB
:1002C000E0ECF0E0908195FFFDCF8AE08093C600DE
:1002D000E0ECF0E0808185FFFDCFC12FD0E080E32E
:1002E0008093C60060E070E0CB0196958795969567
:1002F0008795969587959C01220F331F880F991F2C
:10030000880F991F880F991F820F931F681B790B05
:10031000605DE0ECF0E0808185FFFDCF6093C6007A
:100320009E013695279536952795ABE7B4E10E9457
:100330004E0396958795805DE0ECF0E0908195FF07
:10034000FDCF8093C6009E01ADECBCEC0E944E0335
:10035000FC01F695E795F695E795F695E7959F01EB
:100360000E944E03969587959695879596958795C5
:100370009C01220F331F880F991F880F991F880F28
:10038000991F820F931FE81BF90B9E2F905DE0ECE5
:10039000F0E0808185FFFDCF9093C6009E01ADEC1B
:1003A000BCEC0E944E0396958795969587959695F9
:1003B00087959C01220F331F880F991F880F991F63
:1003C000880F991F820F931FC81BD90BC05DE0ECEB
:1003D000F0E0808185FFFDCFC093C600A6E6B1E0C6
:1003E00090E2E0ECF0E0C6ECD0E0808185FFFDCF4C
:1003F00098839D919111F9CF50E0E0ECF0E080817D
:1004000085FFFDCF80E38093C60060E070E0CB0104
:100410009695879596958795969587959C01220F39
:10042000331F880F991F880F991F880F991F820FFC
:10043000931F681B790B605DE0ECF0E0808185FF25
:10044000FDCF6093C6009A0136952795369527957E
:10045000ABE7B4E10E944E0396958795805DE0EC92
:10046000F0E0908195FFFDCF8093C6009A01ADEC3E
:10047000BCEC0E944E03FC01F695E795F695E795D6
:10048000F695E7959F010E944E0396958795969560
:100490008795969587959C01220F331F880F991F8A
:1004A000880F991F880F991F820F931FE81BF90B64
:1004B0009E2F905DE0ECF0E0808185FFFDCF909372
:1004C000C6009A01ADECBCEC0E944E039695879550
:1004D00096958795969587959C01220F331F880FD7
:1004E000991F880F991F880F991F820F931F481B10
:1004F000590B405DE0ECF0E0808185FFFDCF40933B
:10050000C600AFE6B1E090E2E0ECF0E0C6ECD0E08F
:10051000808185FFFDCF98839D919111F9CFE0EC0B
:10052000F0E0808185FFFDCF8DE08093C600E0EC98
:10053000F0E0808185FFFDCF8AE08093C600DF91E7
:10054000CF911F910895789482E390E026E731E0FF
:10055000E0ECF0E0A6ECB0E07DE06AE011C04081A4
:1005600045FFFDCF5C9359915111F9CF408145FF73
:10057000FDCF7C93408145FFFDCF6C93019719F02F
:10058000E90157E4ECCF299AC0ECD0E006EC10E08A
:100590000F2EFEE2DF2EF02D0F2EFDE0EF2EF02DC0
:1005A0000F2EFAE0FF2EF02D4A99FECF0E94840014
:1005B000888185FFFDCFF801D082888185FFFDCF3E
:1005C000F801E082888185FFFDCFF801F082FFEF1E
:1005D00024E38CE0F15020408040E1F700C00000AF
:1005E0002898E2CFCF93DF93789481E88093C4007A
:1005F0001092C00088E08093C10086E08093C20022
:10060000AFE7B1E095E5E0ECF0E0C6ECD0E080814A
:1006100085FFFDCF98839D919111F9CFE0ECF0E03B
:10062000808185FFFDCF8DE08093C600E0ECF0E097
:10063000808185FFFDCF8AE08093C600DF91CF9156
:1006400008958EE193E00E94F202559A539A239AFC
:1006500081E284BD81E085BD16BC1092B60091EAAE
:100660009093B0008093B1001092B20010926E008F
:100670001092700018BC1092B4001092B300209A2F
:10068000219A2898299856985E9857985F9810BE96
:1006900010927B0083E080937F000895A29FB001B9
:1006A000B39FC001A39F01D0B29F700D811D112483
:1006B000911D0895EE0FFF1F0590F491E02D099410
:0406C000F894FFCFDC
:1006C4000A0D0A0D52656365697665643A200A0D60
:1006D4004F464620094F4E00696E74204952736993
:1006E400676E616C5B5D203D207B002F2F204F46A1
:1006F400462C204F4E2028696E2031302773206FFE
:1007040066206D6963726F7365636F6E647329002D
:100714007D3B002031427974650052656164204458
:100724006174613A002048427974652C2000204CA1
:10073400427974650047656C6164656E210055619A
:0A074400727420646F6E65210000DE
:00000001FF
